:100000002FC149C14CC347C146C145C144C143C1C9
:10001000D8C341C140C13FC14AC43DC13CC13CCE2F
:100020001DCE49CE53CE5DCE6ACE87CE00000000F5
:10003000A60EF9154C1DF22B3E498A6601020304F7
:100040000506070200FFFF00FF000000000000009F
:10005000FF0000000078FF000C3F96FFFF0000004B
:1000600000000000FF00000000FF00146E96FF007B
:100070000000000000FF000000FF001E78FF0000ED
:10008000000000FF0000FF001EFF00000000FF0056
:10009000FF00FF000000FF0000FF00FF0000000065
:1000A0000000000000000000000000000000000050
:1000B0000000000000000000000000000000000040
:1000C0000000000000000000000000000000000030
:1000D0000000000000000000000000000000000020
:1000E0000000000000000000000000000000000010
:1000F0000000000000000000000000000000000000
:1001000000000000000000000000000005070A0ECB
:100110001114181C2024282D32373C41474D5359C7
:100120005F666D747B828A929AA2AAB3BCC5CED751
:10013000E1EBF5FF000000000000000000000000FF
:1001400000000000000000000000000000000000AF
:10015000000000000000000000000000000000009F
:10016000000000000000000000000000000000008F
:100170000005070A0D1013171A1E2125282C3034EC
:10018000383C4045494E52575C60656A6F757A7FCE
:10019000858B90969CA2A8AEB5BBC2C9CFD6DDE434
:1001A000ECF5FFFFFFFFFFFFFFFFFFFFFFFFFFFF7C
:1001B000FFFFFFFFFFFFFFFFFFFFFFFFFFFFFFFF4F
:1001C000FFFFFFFFFFFFFFFFFF0003030304040423
:1001D000050505060607070808090A0B0C0E10128C
:1001E0001416191C1F2225292D3135393D42474C43
:1001F00051565C62686E747D848B9299A1A9B1B9E5
:10020000C2CBD4DDE7F1FBFFFFFFFFFFFFFFFFFFE6
:10021000FFFFFFFFFFFFFFFFFFFFFFFFFFFFFFFFEE
:10022000FFFFFFFFFFFFFFFFFFFFFFFFFFFFFFFFDE
:10023000FFFFFFFFFFFFFFFFFFFFFFFFFFFFFFFFCE
:10024000FFFFFFFFFFFFFFFFFFFFFFFFFFFFFFFFBE
:10025000FFFFFFFFFFFFFFFFFFFFFFFFFFFFFF00AD
:1002600011241FBECFE5D2E0DEBFCDBF10E0A0E677
:10027000B0E0E8E1FEE102C005900D92AA39B107B5
:10028000D9F720E0AAE9B0E001C01D92AF3FB20764
:10029000E1F722D8BFCDB4CE20ED37E0019720F0B2
:1002A000F9013197F1F7FACF08959091F60099236B
:1002B00049F0882321F087E187BBC29A089583E142
:1002C00087BBC2980895815090E0FC01E256FF4F31
:1002D0002491FC01EC5CFE4F3491FC01E653FE4F8F
:1002E000849189BD38BD2BBD8091F200882311F027
:1002F00080E0DBCF0895CF93DF93E091F700F0E04B
:10030000E45CFF4F84918093E2001092CE00109243
:10031000E8001092D8009091FC00992351F0909140
:10032000FB009093D9001092CF001092E90092E068
:1003300001C091E020E030E0682F70E0C92FD0E0EC
:10034000261737070CF036C0A091F700B0E0AA0FCF
:10035000BB1FAC57BF4FED91FC91E20FF31FE4912F
:10036000A9014C0F5D1FDA01A852BF4FEC93A09179
:10037000F700B0E0AA0FBB1FAC58BF4FED91FC9146
:10038000E20FF31FE491DA01A851BF4FEC93A09163
:10039000F700B0E0AA0FBB1FAC59BF4FED91FC9125
:1003A000E20FF31FE491DA01A253BF4FEC932F5FEA
:1003B0003F4FC6CF890F8093E200DF91CF91089520
:1003C000811109C019BC18BC1BBC8091F2008823A4
:1003D00019F081E06ACF77CF089581E08093CD0056
:1003E00093E09093FB008093CB0022E02093E60003
:1003F0009093F7008093FC001092CC001092FA00CA
:100400008093F9001092E3008093F6000895CF9353
:10041000DF931F92CDB7DEB79FEF9BBD90E069835E
:100420003BDF1BBC6981862F90E00F90DF91CF915D
:1004300033CF8091CD008093B9001092CD001092FF
:10044000FE008BE58093BB0080E02FCF8091B90048
:100450008093CD001092C6008091CD00882319F0C2
:100460001092BB0008958091BA008093BB0008955C
:10047000EF92FF920F931F93CF93DF93C82F8B01BF
:100480007B01EE0CFF1CEE0CFF1CD2E3CC2381F0B1
:1004900081E00BDFD9BD18BC1BBCC801FDDE80E0CC
:1004A00004DF19BC18BC1BBCC701F6DEC150EECF7F
:1004B000DF91CF911F910F91FF90EF9008951F93BF
:1004C000CF93DF93C82FD62F12E3CC2311F1809165
:1004D000BB008D131EC081E0E8DE8091F60088230A
:1004E00021F08091E300811103C019BD18BC1BBC31
:1004F0008AEF90E0D1DE80E0D8DE19BC18BC1BBCCE
:1005000087E791E0C9DE8091BB008D1302C0C15026
:10051000DCCFDF91CF911F9108951F93CF93DF938D
:10052000D62F6AE03CDC192F6D2FC9DFC091BB00CC
:10053000CD1310C080E293E0AFDE6C2F812FBFDFC0
:100540008091BB008C1306C080ED97E0DF91CF91C6
:100550001F91A2CEDF91CF911F910895EF92FF924C
:100560000F931F93CF93863018F006E910E002C076
:100570000AEF10E07801EE0CFF1CC82FCC23F1F03D
:1005800019BC18BC1BBCC80187DE81E08EDE8091DF
:10059000CD00882321F08091E50012DF09C0809111
:1005A000FD009091CA002091E40029BD98BD8BBD4B
:1005B000C70172DE80E079DEC150E0CFCF911F919C
:1005C0000F91FF90EF900895EF92FF920F931F937A
:1005D000CF938C017C01F594E794C62FCC2351F086
:1005E00081E063DEC80158DE80E05FDEC70154DED3
:1005F000C150F4CFCF911F910F91FF90EF900895CC
:10060000CF93C82F68E270E082E032DF80EF90E0A5
:1006100043DE64E670E08C2F2BDF1092BC00CF919C
:10062000089586B383FB882780F991E0982780910D
:10063000A400880F892B8093A4009091A300992394
:1006400011F08F7001C081708093A3008091A3008E
:1006500090E008958091BB00803120F48091BB0030
:100660008093BA008091BB008F5F8093BB00909114
:10067000E200891710F01092BB0008958091BB0032
:100680008093BA008091BB00811103C08091E20089
:1006900002C08091BB0081508093BB0008951895E3
:1006A0008EBB6DBB84E28CBB86E28CBBE199FECF36
:1006B0000895CF93DF932091BB008091F700909134
:1006C000CD00880F880F880F979599279795692FE8
:1006D000682B622B6093F8002091CC003091FA00D7
:1006E0009091FB008091CB00330F990F990F932BC2
:1006F000922B8295880F807E892B8093C900409130
:10070000C8005091F6003091F9009091E30080917B
:10071000FC007091E600550F330F330F352B342B4F
:10072000990F990F990F292F232B8295807F982F4E
:10073000922B872F8295880F807E892B8093F400DF
:10074000C091A500D091A600CE0104968F7799277D
:100750009093A6008093A500A3DF8091A5006091EF
:10076000C9008F5F9DDF8091A5006091F4008E5FCE
:1007700097DFCEBB84E18CBB86E18CBBE199FECFD9
:100780008C2F8F5F8EBB84E18CBB86E18CBBE199A3
:10079000FECF8C2F8E5F8EBB84E18CBB86E18CBB41
:1007A000E199FECFCD5FCEBB84E18CBB86E18CBBF3
:1007B000E199FECF8091A5006DE58D5FDF91CF912E
:1007C0006FCF1F920F920FB60F9211245F936F930A
:1007D0007F938F939F93AF93BF9364B175B18091D3
:1007E000AA00813021F5CB0196958795945DE3DAD7
:1007F0006E5F7F4F8091AC008823B9F08091AC0090
:1008000090E08617970728F48091AC008F5F809363
:10081000AC008091AC0090E06817790740F48091BB
:10082000AC0081508093AC0002C06093AC0080911A
:10083000AA008330F9F46B5171408091AB0088239A
:10084000B9F08091AB0090E08617970728F480916B
:10085000AB008F5F8093AB008091AB0090E0681796
:10086000790740F48091AB0081508093AB0002C0C7
:100870006093AB008091AA008F5F8093AA008430C0
:1008800010F01092AA008091AA00823010F48CE03F
:1008900001C08FE887B9BF91AF919F918F917F91F0
:1008A0006F915F910F900FBE0F901F9018951F9240
:1008B0000F920FB60F9211242F933F934F935F9394
:1008C0006F937F938F939F93AF93BF93EF93FF9318
:1008D0008091F500882321F081508093F500EBC4CE
:1008E0008091A8009091A900892B49F08091A800DF
:1008F0009091A90001979093A9008093A80091DEA0
:100900002091B7003091B800892B09F4E9C1203D4E
:1009100087E0380730F42F5F3F4F3093B8002093C3
:10092000B7008091B7009091B800823E24E0920712
:1009300091F42091C70021110EC01092C6001092B0
:10094000E5001092BB001092C50081E08093C000CA
:100950001092BF00B0C43091BF002091B00033238B
:10096000B1F01092BC002111A6C48332910521F48C
:100970008091BF008F5F08C08634910509F09BC449
:1009800081E08093B0008FE08093BF0094C4211178
:100990009CC12091C700222349F0019709F0ABC008
:1009A0008091C0008111A7C086E97BC02091CD0055
:1009B000222309F4A0C0429708F49DC08091C00092
:1009C000811199C08091C100811195C08091BB00B7
:1009D000803508F090C01092A2008091C50081304F
:1009E00009F454C038F0823009F45EC0833009F451
:1009F00065C081C08091C600811121C081E08093D3
:100A0000C50087E18093E7008091FB0089BD18BC99
:100A10001BBC8091F200882311F080E046DC8FEF50
:100A20008093C6008093E5008091C200811104C0CC
:100A30008091C6008093C2001092C3005CC0809178
:100A4000C3009091C400882329F09093C5001092B0
:100A5000C30004C085E0891B8093C5008091C60057
:100A60008F3FD9F08091C600863940F083E08093B3
:100A7000C50086E98093E50026DC3DC08091C60074
:100A80008130C9F582E08093C50035C08091E700D0
:100A900081508093E70081112EC082E08093C500D1
:100AA00081E08093C600E6CF8093C4008091C600A9
:100AB0008639B0F48091C6008F5F09C08093C4006E
:100AC0008091C600823060F08091C6008150809392
:100AD000C6008093E5008091C6008093C20008C0E4
:100AE00084E08093C50080E06BDC87E090E0D4DB9D
:100AF0008091E50065DC8091CD00811135C0809149
:100B0000B7009091B800489779F58091C0008111A5
:100B10002BC08091BB00803190F48091C70081117F
:100B20000EC08091CC00882311F094DD1DC080910F
:100B3000BB00813011F41092BB00A0DD15C0809184
:100B4000BB008B3588F08091FE00811102C080913E
:100B5000630081508093FE00E091FE00F0E0EC56CF
:100B6000FF4F80818093BB008091B7009091B800C7
:100B70008B34910509F075C08091B600823009F57B
:100B80008091B3009091B4000E97D8F48091CD007D
:100B9000882329F08091C000813009F062C0109252
:100BA000C6001092E5001092BB001092C500909113
:100BB000C00081E0282F291B2093C0008093C10032
:100BC00050C08091C00081114CC08091B60081302E
:100BD000A1F42091B3003091B4002E30310568F4B7
:100BE0009091CD0091113DC090E59093BB00809312
:100BF000C10019BC18BC1BBC34C08091BB008B3534
:100C000010F024DC2EC08091BB00803539F41092A6
:100C1000BB0019BC18BC1BBC85E10AC08091BB009D
:100C2000823571F41092BB0019BC18BC1BBC8EE05D
:100C30008093BF001092BD0081E08093B00011C08E
:100C40008091CD0081110DC08091E600882349F08C
:100C50008091BB00803529F08091C700811101C0CF
:100C6000E8DB8091C000811130C08091C700811104
:100C70002CC08091CD0081110FC08091B700909160
:100C8000B800883C910541F48091B600823021F093
:100C90008091BB00803559F48091CD008823A9F064
:100CA0008091B7009091B800843F914071F4109208
:100CB000BB001092C6001092C50019BC18BC1BBC2A
:100CC00081E08093BF001092BD001092A1001092AD
:100CD000A00088E391E09093610080936000E1C2FE
:100CE0001092B0008091BF008823A1F0211531053A
:100CF00059F02831310528F48091BD008F5F809331
:100D0000BD001092BC00C9C28091BC008F5F80936F
:100D1000BC00C3C2232B09F449C18091C7008823BA
:100D200031F01092C6001092E50080E049DB20917E
:100D3000CD008091B7009091B800222309F488C0BB
:100D40001092C500429708F077C08091B6008F5F7F
:100D50008093B6008091B600813009F076C0809112
:100D6000BB0080939F008091BB00803138F480915C
:100D7000C600863919F48FEF80939F008091BB00E5
:100D8000803541F08091BB00813521F08091BB001E
:100D9000823549F41092BB001092C6001092E50013
:100DA00081E08093C1008091C60080939E00809175
:100DB000C00081114AC08091C100811146C080915C
:100DC000C700811142C08091C60081111FC080916F
:100DD000C200811103C081E08093C20081E0809352
:100DE000C30092E09093C4009091C2009093C6001B
:100DF0009093E5009091F60091118093A70089EA05
:100E000093E09093A9008093A80004C01092C600BC
:100E10001092E5008091E5008F3F61F48091FB0026
:100E200089BD18BC1BBC8091F200882371F080E062
:100E30003CDA0BC0C5DA09C01092B6008091F6000A
:100E4000882319F081E08093A7001092C100A9C007
:100E50008831910508F089C08091BB00803541F050
:100E60008091BB00813521F08091BB00823561F417
:100E70008091BB0080939F001092BB008091B600D0
:100E80008F5F8093B6008DC08091BB00811106C03A
:100E90008091B600811102C081E007C08091B60048
:100EA000882329F08091B6008F5F8093B6008091EF
:100EB000C000811176C08091FA00882399F080915A
:100EC000B500882379F08091BB0081110BC080911F
:100ED000C700811166C08091B5008093BB0010925D
:100EE000B5005FC08091BB00803110F58091C700D4
:100EF000811157C08091BB00882391F08091B3008D
:100F00009091B4008B34910558F08091BB00809390
:100F1000B5008091BB008093BA001092BB0041C025
:100F20008091CC00882311F0A9DB3BC093DB39C052
:100F30008091B3009091B4008B34910510F086DA63
:100F400030C08091E6008130D1F3E091FE00EF5F88
:100F5000E093FE0080916300E81788F7F0E0EC561C
:100F6000FF4F80818093BB001CC08B349105B8F487
:100F70008091B600813099F42091B3003091B40093
:100F80002E30310560F49091BB00911108C0909112
:100F9000F200891B8093F2008091F20086D91092B2
:100FA000B6001092B4001092B30077C18091B300E4
:100FB0009091B40001969093B4008093B300892B74
:100FC00031F480E395E79093B4008093B30080916F
:100FD000B3009091B4000F9708F4A6C08091B600BA
:100FE0008530B9F48091CD00882309F49BC08091AD
:100FF000C000811197C08091C700811193C081E02A
:101000008093C7001092C6001092E5001092BB00BA
:1010100038C08091B6008430F9F48091CD00811100
:1010200005C08091C000882309F47CC08091C7006E
:10103000811178C01092C6001092E5001092BB009A
:101040001092C5009091C00081E0282F291B2093A9
:10105000C0008093C10066C080919F0090EB980F04
:10106000923098F49091B600923009F05BC08035D0
:1010700011F481E501C082E58093BB0081E080939B
:10108000C10019BC18BC1BBC4DC08091CD00882389
:1010900009F448C08091C000811144C08091C7000C
:1010A000811140C08091B600833049F480E580937F
:1010B000BB0081E08093C10019BC18BC1BBC8091AF
:1010C000B600823079F580919F008F3FC9F48091FE
:1010D000E600882311F0ADD925C08091C200863981
:1010E00039F08091A2008093C6008093E50004C08F
:1010F0001092C6001092E5008091E50061D912C0FF
:1011000086E98093C6008091C6008093E50058D997
:1011100080919E008093A20089EA93E09093A900B9
:101120008093A8001092B6008091CB008230E8F145
:101130008091CD008823E1F08091E50088588737C1
:10114000A0F58091A0009091A10001969093A1003C
:101150008093A0002091B1003091B2002817390788
:1011600020F58EE78093C6008093E500ACD81DC0C3
:101170008091BB008031C8F4E091BB00F0E0E25305
:10118000FF4F80818F3F89F48091A0009091A10052
:1011900001969093A1008093A0002091B10030911E
:1011A000B2002817390708F469DA8091CD00882346
:1011B00091F08091C600823070F08091C60086392F
:1011C00050F48091B3009091B4008C34910518F0E4
:1011D00081E08093C300809160009091610000974E
:1011E00029F00197909361008093600080916000E6
:1011F00090916100892BD1F59091BB008091CD0039
:10120000811104C081E0913041F408C09091E50063
:1012100081E0913019F09F3F09F080E02091AC000F
:1012200030E0811103C08EE190E002C08CE190E0DB
:101230002817390734F480919D008F5F80939D00BB
:1012400004C010929D001092AE0080919D008830E5
:1012500068F081E08093AF008093AE0010929D0013
:1012600088E391E090936100809360008091AE00EC
:10127000882399F080919B0090919C000196909317
:101280009C0080939B00843F914039F481E08093DF
:10129000AD0010929C0010929B001092B80010922A
:1012A000B70080919A008F5F80939A00837019F441
:1012B00086B1886486B9FF91EF91BF91AF919F91FC
:1012C0008F917F916F915F914F913F912F910F90EF
:1012D0000FBE0F901F90189517BA88E088BB85BB8A
:1012E00083E187BB81EA8ABD81E083BF80BF80E65E
:1012F0008CBD8FEF8DBD8CE087B9A29A87EC86B943
:10130000479A85B7877E806185BFF8948BB78F7DBC
:101310008BBFA89584B7877F84BF81B5886181BD65
:1013200011BC5BD81092A6001092A5000091A500F8
:101330001091A6000038110508F02CC5C80162D52F
:10134000F82E8093F800C80101965CD5D82F8093C1
:10135000C900C801029656D5C82F8093F400C80171
:10136000039650D58D3539F00C5F1F4F1093A600B2
:101370000093A500DBCF8F2D87708093BB008F2D4E
:101380008695869586958F708093F700FF1CFF24C5
:10139000FF1CF092CD008D2F81708093CC00D1FB8B
:1013A000882780F98093FA008D2F8695869587701F
:1013B0008093FB00D295D695D770D093CB008C2F1D
:1013C00081708093C800C1FB882780F98093F60064
:1013D000C2FB882780F98093F900C3FB882780F936
:1013E0008093E300C4FB882780F98093FC00C295BA
:1013F000C695C370C093E6008091F9008093F20017
:101400008AEF90E0FFD49FEF980F9E3F10F48093F7
:10141000620071D7E091CB00F0E0EE0FFF1FE45DBA
:10142000FF4F859194919093B2008093B100809189
:10143000C800882359F08091CD00811107C08091A8
:10144000FF00811105C006D934D902C01092BB003B
:101450008091BB0081110CC08091CD00811104C02E
:101460008091C800811104C060E570E082E000D87E
:101470001092FF008AEF8093F30089E18093F500DA
:10148000F894A89581B5886181BD80E481BD789488
:10149000812C912C312CC1E0DFE058E2552E1FEF5A
:1014A00068E3C62EDD24D3947CEFE72E7AE0F72E96
:1014B000E5E0AE2EB12C44244A948091BF00811106
:1014C0008FC28091C0003816B1F03090C00019BCB6
:1014D00018BC1BBC6BE470E084E0CAD71092C1005A
:1014E0008091C000882329F08091BB008093F30095
:1014F00002C04092F3008091C700981669F0909066
:10150000C7006CE370E082E0B3D78AEF90E0C4D606
:101510006BE470E083E0ACD79091BB008091F30066
:10152000981709F405C18091BB00803188F520919E
:10153000BB00822F90E0FC01E852FF4F30813093D6
:10154000E400FC01E851FF4F30813093CA00FC01F8
:10155000E253FF4F80818093FD008091FD009091C8
:10156000CA003091E40039BD98BD8BBD211106C081
:101570008091F200882311F081E004C08091F30093
:10158000811101C092D68091BB008093F300D0C03E
:101590008091BB008093F30019BC18BC1BBC8091E8
:1015A000BB00803579F480E991E076D61092C100D5
:1015B0008091BB00803509F0BBC08091AC0060E534
:1015C000ACD7F6CF8091BB00813579F48AEF90E0FB
:1015D00063D61092C1008091BB00813509F0A8C08C
:1015E0008091AB0061E599D7F6CF8091BB00823541
:1015F00071F48AEF90E050D61092C1008091BB0048
:10160000823509F095C062E58CE087D7F7CF8091ED
:10161000BB008B3549F48091BB008B3509F088C045
:1016200069E28EE0F4D6F7CF8091BB008C35E1F40F
:101630008091BB008C3509F07BC008E08091BB0035
:101640008C3511F008E00BC068E284E1E0D601506F
:10165000A9F7F8CF60E588E2DAD6015049F3809126
:10166000BB008C35B9F3E4CF8091BB008D3541F5DB
:101670008091BB008D3501F504E08091BB008D3574
:1016800011F00AE014C019BC18BC1BBD85E090E045
:1016900003D619BD18BC1BBC81E490E0FDD50150F8
:1016A00061F7EFCF88E490E0F7D5015009F380911E
:1016B000BB008D35B9F3DCCF19BC18BC1BBC38C0DE
:1016C0008091BB008E35C1F48091BB008E3581F5D1
:1016D0008CE291E0E1D56DE78DE799D66DE78DE776
:1016E00096D60FE08091BB008E3571F784E690E0CE
:1016F000D3D50150B9F7E8CF8091BB008F35C1F445
:101700008091BB008F35A1F48CE291E0C5D560EFEC
:1017100080EF7DD660EF80EF7AD604E68091BB0043
:101720008F3571F784E690E0B7D50150B9F7E8CF6F
:101730008091AF00882309F445C08091CD008823B3
:1017400069F18091E5008823D1F1813011F08F3F5C
:1017500061F487E08093E50088E000D71092C6002E
:101760001092E5001092C50012C083E0F7D6809178
:10177000E5008A3050F090E0880F991F880F991F7C
:10178000B5012DD36093E50002C0C093E5008091C0
:10179000E50016D68AEF90E07FD511C08091BB009E
:1017A000882369F08091BB00813011F488E001C08A
:1017B00083E0D4D68091BB00803108F45FD71092CB
:1017C000AF0034C08091AD00882381F18091F60094
:1017D000882351F18091F2008823A9F08091CD00F7
:1017E000882321F08091E500811108C08091CD000F
:1017F000811109C08091BB00882329F062E084EF49
:1018000091E0E2D611C080E050D584EF91E044D55C
:1018100081E04BD584EF91E03FD580E046D584EF61
:1018200091E03AD581E041D51092AD008091CB0096
:101830008130C9F59091AB0080916200981798F1C2
:101840008091A8009091A900892B69F58091CD0025
:101850008823C1F08091E5009FE8980F9E3818F525
:10186000282F30E066E09BD2A901481B5109CA012C
:10187000413751050CF480E78093E5008091E50045
:101880009FD509C08091BB00882369F08091BB007F
:10189000803148F4F3D6F092A900E092A80063E00A
:1018A00084EF91E091D68091AE00882329F034EE48
:1018B000632E37E5732E04C026E3622E77247394DB
:1018C0008091CD00811104C08091BB00882349F034
:1018D0008091CD00882309F45AC08091E5008111E0
:1018E00056C09FD6892B09F052C08091B3009091C9
:1018F000B4006816790608F04AC08091AC008E31B9
:1019000030F48091F200882311F080E0CED481E0A1
:1019100090E0C2D41092B4001092B3001092A900CB
:101920001092A800F894A89584B7877F84BF81B5EA
:10193000886181BD11BC789437981092B8001092DC
:10194000B7006FD6892B21F080E190E0A5D4F9CFC4
:101950008BB780628BBF85B7806285BF85B784688F
:1019600085BF8B7F85BF889585B78F7D85BF8BB7FA
:101970008F7D8BBF8CE087B9A29A87EC86B9F894EB
:10198000A89581B5886181BD80E481BD78948091FE
:10199000A700882309F491CD1092A7008091E5005B
:1019A000882309F48ACD8F3340F0813720F08F3FB0
:1019B00021F003E003C002E001C001E08CE291E00D
:1019C0006BD481E072D48FEA90E066D480E06DD46D
:1019D000013019F08FEA90E05FD4015091F76DCD9E
:1019E0008091BD00881581F08090BD008091BD0080
:1019F000882351F084E189BD18BC1BBC84E690E0CB
:101A00004BD419BC18BC1BBC9091BF008091BE0088
:101A1000981709F4A3C18091BF008093BE00109273
:101A2000BC008091BF00873109F47CC0E0F48E30A7
:101A300009F448C028F4813059F1833091F1E1C0B4
:101A40008F3009F45AC0853109F0DBC080E991E09C
:101A500023D481E0D5D58091BF008F5F8093BF00F4
:101A60001092BD0078C1883209F475C138F488310C
:101A700009F467C0893109F471C0C3C0843609F420
:101A800079C0853609F482C0893209F0BAC08EC0A7
:101A900080E991E001D481E0B3D58091BF008F5FF0
:101AA0003CC18091BD00882359F08091BD008930F0
:101AB00038F48091BD0081708C278093CD00F9D5DA
:101AC00082E039C18AD4F5D58091F9008093F20083
:101AD00012D48CE3809362006CE38AEFE1D5E0914D
:101AE000CB00F0E0EE0FFF1FE45DFF4F8591949176
:101AF0009093B2008093B1002CC11092BF0068E2B5
:101B000070E085E0B5D41092C6001092E500109206
:101B1000BB008091CD00882309F41DC18091C600CF
:101B20004FD419C18091BD00882351F28091BD002E
:101B300081708C278093F9008091F9008093F200E6
:101B4000BECF8091BD00882339F08091BD008170A7
:101B50008C278093E300ADD583E0EDC08091BD007C
:101B6000882309F4F6C08091BD0081708C27809392
:101B7000F600EEC068E270E083E07AD419BC18BCCD
:101B80001BBDD092A900C092A800E5C019BC18BC2A
:101B90001BBC8091A8009091A900892B11F5609140
:101BA000AB00609362008AEF7BD51BC08091BD00C3
:101BB0008823B9F08091BD00873098F48091BD00F2
:101BC0008F5F8093CB0075D5E091CB00F0E0EE0FF6
:101BD000FF1FE45DFF4F859194919093B200809335
:101BE000B1008091CD00882321F084E009D585E003
:101BF00003C088E005D589E08093BF008093BE00D4
:101C0000AAC08091CD008823C1F18091BF008530AA
:101C1000A1F0863079F1843009F09DC08091BD003B
:101C2000882309F499CF8091BD00883008F094CFC3
:101C30008091BD008093FB003CC08091BD0081304D
:101C400019F41092CB0013C08091BD00823009F4CA
:101C500060C08091BD00833059F466C0882341F094
:101C60008091BD0081708C278093FC0044D321D5E6
:101C700084E061C08091BD0060C0E091BF008E2F04
:101C800090E0FC013497E730F10508F064C0E15FB3
:101C9000FF4F8091BD000994882309F45DCF8091A6
:101CA000BD008D3008F058CF8091BD0081508093E9
:101CB000F70021D350CF882339F08091BD00817087
:101CC0008C278093CC00F5D485E035C0882339F08B
:101CD0008091BD0081708C278093FA00EAD486E061
:101CE0002AC0882351F08091BD00883030F4809163
:101CF000BD008093FB00FFD2DCD487E01CC08130A4
:101D000021F41092CB00D5D415C08091BD00823053
:101D100039F4C093CB00CDD484E68093BF001BC0C0
:101D20008091BD00833031F468E270E0A1D350921D
:101D3000BF0011C088E064D40EC0882351F08091A8
:101D4000BD00843030F48091BD0081508093E60066
:101D5000B0D4D093BF001092BD00AFCB8091BD0036
:101D6000882321F08091BC008E3770F48091BF00F1
:101D7000843609F4A2CB8091BD0081119ECB809165
:101D8000BC008C3D08F499CB8091BF008F5F80939D
:101D9000BF0093CB1092A6001092A5002DCB991BEB
:101DA00079E004C0991F961708F0961B881F7A9552
:101DB000C9F780950895AA1BBB1B51E107C0AA1F54
:101DC000BB1FA617B70710F0A61BB70B881F991FDC
:101DD0005A95A9F780959095BC01CD01089597FB80
:101DE000072E16F4009406D077FD08D0E4DF07FC38
:101DF00005D03EF4909581959F4F0895709561951B
:101E00007F4F0895E199FECF9FBB8EBBE09A992743
:081E10008DB30895F894FFCF93
:101E180038013C059B0095008C00800071005F0034
:101E28004A0044009C0097008F00840076006500FB
:101E3800510046009D009900920088007B006B00CD
:0A1E4800580048005B5C5D5E5F001F
